:105E330001130000090101240200000301FA040018
:105E4300FA0500030A0A5A0B001E0C00FA0D0003A0
:105E53000E00030F0164100096120132130AFA14A4
:105E6300010215000217010A1801FA1905321A0175
:105E73000A1B01FA1C05321FFFFF20FFFF23011E2F
:105E83002400642A00FA2B00FA2C50782D003D2EB2
:105E930000462F001E3000643250783432FA350148
:105EA30064360164370150380A643C00643E003CA8
:105EB3003F000140FFFF411450420A5A430AC844BD
:105EC30005324500B44600FA4701484802034C0036
:105ED300FA4EFFFF500404510596520A32530B4603
:105EE300540A96560102570546580002590A465A63
:105EF30032FA5B010A5C0A325E000A5F00FE61FF50
:105F0300FF6402106600026701016A0A3C6B00002D
:105F13006C32967300007400007801327901327E8E
:105F2300FFFF81FFFF84FFFF8500AF86000187002D
:105F3300FA89010A8A00009900009D0A969E0001D1
:105F43009FFFFFFAFAFA000009010124020000038F
:105F530001FA0400FA0500030A0A5A0B001E0C009A
:105F6300FA0D00030E00030F0164100096120132B4
:105F7300130AFA14010215000017010A1801FA198D
:105F830005321A010A1B01FA1C05321FFFFF20FF0D
:105F9300FF23011E2400642A00FA2B00FA2C5078F8
:105FA3002D003D2E00462F001E3000643250783401
:105FB30032FA350164360164370150380A643C0013
:105FC300643E003C3F000140FFFF411450420A5A27
:105FD300430AC84405324500B44600FA4701244841
:105FE30002024C00FA4EFFFF500404510596520A78
:105FF30032530B46540A9656010157054658000181
:10600300590A465A32FA5B010A5C0A325E000A5F99
:1060130000FE61FFFF6402106600026701016A0A65
:106023003C6B00006C329673000074000078013200
:106033007901327EFFFF81FFFF84FFFF85FFFF862B
:10604300FFFF87FFFF8901028A00009900009D0A74
:10605300969E00019FFFFFFAFAFA0065006F007930
:106063000083008D009700A100AC00B600C000CAF9
:1060730000D400DE00E800F2005B0063006A0072F7
:10608300007A008200890091009900A100A800B065
:1060930000B800BF00C700CF00D600DF00E600EE67
:1060A30000F600400046004C00520059005F0065B6
:1060B300006B00710077007D00830089008F0095DD
:1060C300009C00A200A800AE00B400BA00C000C645
:0E60D30000CC00D200D900DF00E500EB00F1A8
:1035E700900049E0D3940440149007BAE0FEA3E0AA
:1035F700FF905E3512621AE493F59980129007BA2C
:10360700E0FEA3E0FF905F4912621AE493F59990F8
:1036170007BAE0FEA3E0FF905E33E493FC740193E6
:10362700FDEFB50507EEB50403754D009007BA1217
:1036370062012285F97285FA737E017F00E57312B4
:1036470061F3E5722FFF50010E8E598F5A900013C8
:10365700E0FCA3E0FDEF2DFDEE3CFC8C5B8D5C22D6
:1036670075A71085F97285FA737E017F00E57312DD
:1036770061F3E5722FFF50010E8E598F5A9000DCCF
:10368700E0B40210AC2CAD2DEF2DFDEE3CFC8C5BB5
:103697008D5C8016AE59AF5A900013E0FCA3E0FD95
:1036A700EF2DFDEE3CFC8C5B8D5C22AE59AF5A745E
:1036B7000A8E048F05FF1261E38C5B8D5CAE59AFF8
:1036C7005A740A8E048F05FF12620E8C598D5AE5C3
:1036D7005A45596013740AC3955AFFE49559FE8EEB
:1036E700598F5A785B126247E572A85BB80015D309
:1036F700955C4010E572C3955CFFE4955BFE8E5BBD
:103707008F5C8010E5722424C3955CFFE4955BFE13
:103717008E5B8F5CAE5BAF5C74236F4E6006742468
:103727006F4E701AAE5BAF5C74236F4E7005757287
:10373700018003757202755C22755B0080037572E8
:10374700002290008AE0B40104C2108002D21090D7
:10375700008BE0B40104C2118002D2119000C8E0CE
:1037670075F0DCA4FFAEF0740A8E048F05FF1261BA
:10377700E39007B0ECF0A3EDF0A20D401674038CB4
:10378700068D071261F374011200399007AEEEF04F
:10379700A3EFF07E017F00900086E01261F39000B6
:1037A700C9E08E048F05FF1261E3740AFF1261E31B
:1037B7008D5F9000D2E075F0DCA4FFAEF0740A8E46
:1037C700048F05FF1261E39007B4ECF0A3EDF090CE
:1037D70000D4E060139000D4E0F5F0741684FF7E07
:1037E70000EF9007BEF0800674649007BEF090006B
:1037F700CAE090006EF0900114E0900058F090003D
:10380700A3E090005AF09000CCE090005BF09000AD
:1038170078E090005CF09000FEE0900061F074E3C7
:1038270090006DF09000B3E0B40B0874E390006D66
:10383700F0805A9000B3E0B419129000C9E090608C
:103847004812008CE49390006DF080419000B3E043
:10385700B41E129000C9E090606612008CE4939049
:10386700006DF080289000B3E0B428129000C9E002
:1038770090609012008CE49390006DF0800F9000A0
:10388700B3E0B446089000AAE090006DF090007194
:10389700E0FE9000B0E0B50633900073E0FE9000C4
:1038A700CEE0B50627900072E0FE9000DCE0B5069A
:1038B7001B900075E0FE900083E0B5060F90007442
:1038C700E0FE9000BEE06E7003023A13900049E0FC
:1038D700C39405500874029000FFF080149000DC38
:1038E700E0600874089000FFF08006740A9000FFFB
:1038F700F0900083E0B4010674009000E9F09000B6
:1039070083E0B4020674009000CEF0900083E0B428
:10391700030674009000DBF09000CEE0D3940140E2
:10392700147418900101F074009006C8F0740090A8
:1039370006C9F0800C7400900101F074189006C855
:10394700F09000B0E06014741A900097F074009043
:1039570006D0F074009006D1F0800C7400900097A8
:10396700F0741A9006D0F09000B0E0B40214741905
:10397700900098F074009006CCF074009006CDF09B
:10398700800C7400900098F074199006CCF09000A9
:10399700DCE0700E74059006DCF074069006E0F02B
:1039A700801874009006DCF074009006DDF0740057
:1039B7009006E0F074009006E1F0D2269000B0E0A7
:1039C700900071F09000DCE0900072F09000CEE083
:1039D700900073F09000BEE0900074F0900083E0D8
:1039E700900075F0900083E0900059F09000BEE0E1
:1039F70090005DF09000DCE090005EF09000B0E099
:103A070090005FF09000CEE0900060F09000E6E05C
:103A1700B4011790001F740FF0A374FFF0900021FA
:103A2700E4F0A3F074029000E6F09000E6E0B4033F
:103A370041900021E0FEA3E0FF90001FE0FCA3E01F
:103A4700FD12623F74101261F37408120039EF908F
:103A5700006AF0EF700674FF90006AF0740090003F
:103A6700E6F0900020E090006BF090001FE09000DF
:103A77006CF0900077E090003BF090003BE0241260
:103A870090003CF090003CE0D39424400B90003C25
:103A9700E0C3942490003CF090003FE4F090003B9A
:103AA700E06423600790003BE0B4242090003BE0F3
:103AB700B42306740290003FF090003BE0B4240664
:103AC70090003F7401F090003B7401F0900040E4D7
:103AD700F090003CE06423600790003CE0B42420B1
:103AE70090003CE0B423067402900040F090003C44
:103AF700E0B424069000407401F090003C7401F09B
:103B0700900077E0FE9000DAE02E900042F09000FF
:103B170042E064126007900042E0B424069000423D
:103B2700E004F0900042E064116007900042E0B4C6
:103B37002306900042E014F0900042E0D394244022
:103B47000B900042E0C39424900042F0900042E0C2
:103B5700D39412400D900042E0C39412900043F0BA
:103B6700800A900042E02412900043F075501290B2
:103B770000BDE090003DF090003DE075F01284AF8D
:103B8700F07E00EF4E700690003DE004F090003D9F
:103B9700E00475F01284AFF07E00EF4E70069000DF
:103BA7003DE014F090003DE0B4490690003D7401FB
:103BB700F090003DE0D39424400F90003DE0C39483
:103BC7002490003DF0D2208002C22090003DE0D337
:103BD7009412400D90003DE0C3941290003EF08097
:103BE7000A90003DE0241290003EF022C293C29456
:103BF700C291C292C287C290E5B554EFF5B5E5B55B
:103C070054DFF5B5C296C295C2A0C297C2A2C2A19F
:103C1700E5B554BFF5B5E5B5547FF5B5E5B554FB46
:103C2700F5B5C212755D469000C0E07005756C026F
:103C37008003756C0375540075530090000874FF7A
:103C4700F0A374DCF0C217C21974C8900033F07483
:103C5700C8900037F0755200755100C20D754600C7
:103C6700E56EB40903756E00756200900015E4F007
:103C7700A3F0756F10C215C2169007B0E0FEA3E05F
:103C8700FF74031261F374011200399007AEEEF06E
:103C9700A3EFF0C20275560075550090000CE4F0D2
:103CA700A3F0C227755800755700900082E075F0A1
:103CB70032A4FDACF090001DECF0A3EDF0C237226A
:103CC70085F97285FA737E017F00E5731261F3E56A
:103CD700722FFF50010E8E598F5AAC5BAD5CEF2DE2
:103CE700FDEE3CFC8C5B8D5CD293D294E55CF5FBDE
:103CF700E55BF5FCE55CF5E9E55BF5EA9000BEE020
:103D0700B40314D291D292E55CF5EBE55BF5ECE5F3
:103D17005CF5EDE55BF5EE2275A71085F97285FA7E
:103D2700737E017F00E5731261F3E5722FFF500187
:103D37000E8E598F5A7E017F769000FBE01261F359
:103D4700AC59AD5AED2FFFEC3EFE8E5B8F5CE55C08
:103D5700F5FDE55BF5FE90006EE4F075A7007412C3
:103D6700900045F02285F97285FA737E017F00E5A0
:103D7700731261F3E5722FFF50010E8E598F5A901F
:103D870007B0E0FCA3E0FDEF2DFDEE3CFC8C5B8D66
:103D97005CE55CF5FDE55BF5FE220563229000BE60
:103DA700E0B403539000DCE0B4012EA2D8B3400482
:103DB700C293C287A2D9B34004C294C290A2DAB315
:103DC7004008C291E5B554EFF5B5A2DBB34008C290
:103DD70092E5B554DFF5B5801CA2D8B34002C29373
:103DE700A2D9B34002C294A2DAB34002C291A2DBC5
:103DF700B34002C292801EA2D8B3400AC293900079
:103E0700DCE06002C287A2D9B3400AC2949000DC0A
:103E1700E06002C290A2DCB34004C296C29575D896
:103E2700402285A77175A710A2D8B34002C287A206
:103E3700D9B34002C290A2DAB34006E5B554EFF514
:103E4700B5A2DBB34006E5B554DFF5B5A2DCB34058
:103E5700089000CAE090006EF075D8408571A722DF
:103E6700900047E4936406600280FE74C89007B62A
:103E7700F8E4F0E8A3F075B50075840175A700753F
:103E8700FFA0900041E4F075C91075A70F75A1C791
:103E970075A70075D90075CE0C75A70F75F1FE755E
:103EA700F2FF75F30775F47875A4BA75A5FF75A6C3
:103EB7000775AE0075AFFF75D48175D5FF75D6FF51
:103EC70075D7FF75A70075A20175A14775F8097524
:103ED700D80075D90475DA0975DB0975DC0975DD54
:103EE7000975DE0975D84075A71075D80075D9040E
:103EF70075DA0975DB0975DC0975DD0975DE097584
:103F0700D84075A70075E60875E71075BC0175BE42
:103F17000475BD6C75BE0775BDA075BE0875BD017E
:103F270075BC0075BB1875BC2075BA0875E8807537
:103F3700D11375A70F75E10575E20075C740123BF0
:103F4700F3759700759780740A1261D37597C0E56A
:103F5700975420700280F8758F0275A700D2AF754D
:103F6700980075A90C75A70F75AB4375ADFB75ACBC
:103F77001E75A71075C91875CA0075CB0075C804DA
:103F870075A700758912758E04758C00758A00C235
:103F9700A9D28C758D00758B00D2ABD28E75EF06CA
:103FA70075D944C29974C8F5097508001200E375FC
:103FB700B5001204E374639007B6F8E4F0E8A3F0E1
:103FC70012036F74C89007B6F8E4F0E8A3F07464BE
:103FD700F5097508001200E3900059E0900083F09E
:103FE700C21D900083E0D3940340067400900083C1
:103FF700F0900083E0905A4BF82828738028A2B4E9
:104007004002D21D802075A70F75F30F75A700A278
:10401700A34002D21D800F75A70F75F31775A70070
:06402700A2A44002D21D1C
:0C5A4B0002400302400502400D02401E14
:10402D00A21DB34066757208E572D3940E5020E55B
:10403D00729007B6F8E4F0E8A3F012023E7464F54E
:10404D00097508001200E37872740126F650D974D0
:10405D00029000BFF0900083E0D3940340067400FB
:10406D00900083F0900083E0905A57F828287380D1
:10407D001674009000E9F0800E74009000CEF08070
:07408D000674009000DBF057
:0C5A570002407C02407E02408602408E2D
:10409400D21C8064757201E572D394075020E572D6
:1040A4009007B6F8E4F0E8A3F012023E7464F50950
:1040B4007508001200E37872740126F650D9740171
:1040C4009000BFF0900083E0D39403400674009006
:1040D4000083F0900083E0905A63F82828738016D8
:1040E40074009000E9F0800E74009000CEF0800619
:0640F40074009000DBF0F7
:0C5A63000240E20240E40240EC0240F489
:1040FA00C21C900058E0900114F0900059E0900022
:10410A0083F090005AE09000A3F090005BE09000EA
:10411A00CCF090005CE0900078F090005DE09000B8
:10412A00BEF090005EE09000DCF090005FE090004E
:10413A00B0F0900060E09000CEF0900061E0900056
:10414A00FEF09000C9E07006740A9000C9F0900071
:10415A00AAE0700674E39000AAF09000B0E0049020
:10416A000071F0123749E5B54401F5B574069000BF
:10417A0047F07401900048F0740390004AF0740507
:10418A0090004BF0741490004CF0740590004DF0C0
:10419A00900049E0B40406740490004DF074009055
:1041AA00004EF07400900053F07400900054F074C4
:1041BA0001900055F07400900056F074FF9000577B
:1041CA00F0743390014DF0743690014EF0742D90D6
:1041DA00014FF07432900150F07420900151F07444
:1041EA0034900152F07443900153F0747990015461
:1041FA00F0746C900155F07420900156F074209080
:10420A000157F07420900158F07420900159F0740D
:10421A002090015AF0742090015BF09000E5E09044
:10422A00006AF090009CE090006BF090009DE09096
:10423A00006CF0A2B6B3920EA2B3B3920FA2A4B3CB
:10424A009223A2B4B39224A2A3B39225900066E467
:10425A00F0756E00743A900776F074FD900777F067
:10426A00900067E4F09007B0E0FEA3E0FF74031249
:10427A0061F374011200399007AEEEF0A3EFF07506
:10428A006D01900045E4F0C222756200C213D21497
:10429A00C202757000C229D203C22AD204C22BD22A
:1042AA0005C22CD206C22DD207C22ED208C22FD2E4
:1042BA0009C230D20AC231D20BC232D20CC21EC2D9
:1042CA001FC220C221C22612009E755E00756A00B6
:1042DA0075600075643275650075660075670075EE
:1042EA006800756900900015E4F0A3F0756B00D2C0
:1042FA00B2D2A4D2B0D2B1D2A3D2A7D2A6D2A5D2D8
:10430A00B7900082E0D394FA400674FA900082F0E3
:10431A007E017F0090006CE01261F390006BE02F49
:10432A00FF50010E90001FEEF0A3EFF0EFD394FFC1
:10433A00EE940F400790001FE4F0A3F090006AE0AB
:10434A00700674FF90006AF074009000A9F0900063
:10435A00BFE0D39402400674019000BFF09000C001
:10436A00E07005756C028003756C039000C1E0D3A0
:10437A009401400674009000C1F09000C7E0C39415
:10438A000A5006740A9000C7F09000D1E0700674D3
:10439A00019000D1F09000D1E0B4FF0674FE9000C5
:1043AA00D1F09000D8E0D394FE400674FE9000D875
:1043BA00F09000FEE0D39402400674019000FEF0F3
:1043CA00900114E0D3940140067401900114F07432
:1043DA00019000DEF074019000DFF074009000E6B6
:1043EA00F07400900102F07400900106F0742990B4
:1043FA0006BCF0742A9006C0F074179006C4F074D4
:10440A001B9006D4F0741C9006D8F0D29C9000B190
:10441A00E0D39404400674049000B1F09000E3E005
:10442A00D39404400674049000E3F0E56FD394102B
:10443A004003756F109006BDE0D3940C40067400DB
:10444A009006BDF09006C1E0D3940C40067400902B
:10445A0006C1F09006C5E0D3940C4006740090069D
:10446A00C5F09006C9E0D3940C400674009006C9C2
:10447A00F09006CDE0D3940C400674009006CDF07F
:10448A009006D1E0D3940C400674009006D1F090C7
:10449A0006D5E0D3940C400674009006D5F0900639
:1044AA00D9E0D3940C400674009006D9F09006DD4A
:1044BA00E0D3940C400674009006DDF09006E1E02B
:1044CA00D3940C400674009006E1F0D2EC75CF014B
:1044DA00A298B34005C298120616E54D6006A29945
:1044EA00B3B340028005C299120AB4E54E64016072
:1044FA0005E54EB4040280D5C28E7E107F00E563C6
:10450A001261F3E58D75F010A4FDACF0EF2DFDEE10
:10451A003CFCE58B75F01084FF7E00ED2FFFEC3E2E
:10452A00FE8E538F54D28E9000A3E060099000A3B0
:10453A00E0C3943D4002805C900017126201900033
:10454A0017E0FEA3E0FF900019E0FCA3E0FDEFB541
:10455A000542EEB5043EB21BA20DB3401975E70041
:10456A00A21BB34008E5B54404F5B58006E5B55489
:10457A00FBF5B575E710900019E0FEA3E0FF900087
:10458A001BE0FCA3E0FDEF2DFDEE3CFC900019ECD6
:10459A00F0A3EDF09000B0E060099000B0E0C394A1
:1045AA00034002806F1229C0A20DB3500990006621
:1045BA00E0C3941C4002800690009AE0F545E54568
:1045CA0075F005A4FFAEF09007B8EEF0A3EFF090F7
:1045DA000087E0C395604007E55EC3955F5007908A
:1045EA0007B8E4F0A3F0AE2EAF2F9007B8E0FCA313
:1045FA00E0FDEFD39DEE9C4004C2A1800B900066C3
:10460A00E0C3942A5002D2A19000B0E0B40205A2FD
:10461A00A1B392A29000B0E0B4031C122ADBAE2E22
:10462A00AF2F9007B8E0FCA3E0FDEFD39DEE9C40CE
:10463A0004D2A18002C2A190008BE06009A2B3302B
:10464A000F01B3B340028039A2B3300F01B3403136
:10465A00A2B3301101B3401C9000BEE0B40306A21D
:10466A001EB3B3400280067404900045F0D21EA225
:10467A0011B3920FA211B330B301B34004A2119245
:10468A000FA2B6300E01B35003024D08A2B6300E87
:10469A0001B35003024D08A2B6301001B350030211
:1046AA004B2C756D009000A3E0B43D1975E700A28C
:1046BA0010B34008E5B554FBF5B58006E5B54404EA
:1046CA00F5B575E710055DA212B3B35013AE53AF3B
:1046DA0054900008E0FCA3E0FDEDC39FEC9E40036C
:1046EA00024836E56CB4032EA227B34022E55DB436
:1046FA002303756C01E55DC394235006900045744D
:10470A0001F0E55DD3942340067402900045F075EC
:10471A005D01D227805AE56CB40206756C01755D9D
:10472A0023E55DB42305755D018045900045E07081
:10473A0030E55DC3942350069000457401F0E55DB1
:10474A00D3942340067402900045F0E55DC3942398
:10475A005002D222E55DD394234002D222C296C2ED
:10476A00959000C0E0B40105123BF38003755D012A
:10477A00AE55AF56AC53AD54EF2DFDEE3CFC740272
:10478A008C068D071200398E558F569000A3E06073
:10479A00099000A3E0C3943D40028043900017E0D3
:1047AA00FEA3E0FF9000A3E08E048F05FF1261E3F1
:1047BA0074018C068D0712003990001BEEF0A3EFEE
:1047CA00F090001BE0F8A3E0900019C8F0A3C8F02D
:1047DA00900017E4F0A3F0C21BE5B554FBF5B5A2AF
:1047EA00B4B34002C224A2A4B34002C223A2A3B318
:1047FA004002C225A222B34002C222A21EB3400630
:10480A00A220921F8002B21F90008BE06012E56C1A
:10481A00700EA21EB35009A21F302001B3B340028A
:10482A0080067405900045F0C21E803AAE55AF5618
:10483A00AC53AD54EF2DFDEE3CFC74018C068D0794
:10484A001200398E558F56E56CC39402500DAC5345
:10485A00AD547488C39D74139C40028009123BF3C3
:10486A007406900045F0E55DB42312740390004588
:10487A00F0D2229000C0E0B40103123BF3AE57AF6E
:10488A0058AC53AD54EF2DFDEE3CFC8C578D58AE11
:10489A0053AF54EFD39DEE9C401190000FE0FAA362
:1048AA00E0FBEBC394E8EA94034002800690000F11
:1048BA0012620190000CE0FEA3E0FFAC53AD54EF8E
:1048CA002DFDEE3CFC90000CECF0A3EDF09000C046
:1048DA00E0B40118AE53AF5474051261F3740112B7
:1048EA000039900008EEF0A3EFF08011AE53AF54F8
:1048FA0074021261F3900008EEF0A3EFF0C28E7515
:10490A008D00758B00756300755401755300D28E46
:10491A00E55D240875F00984AFF07E00EF4E7075EE
:10492A0090000CE0F8A3E090000AC8F0A3C8F09049
:10493A00000AE0FEA3E0FFEF4E600B7C7A7D4C128A
:10494A0060E18E518F5290000CE4F0A3F0AE51AFAB
:10495A00527428BE00039F5010E5622FFF50010ECB
:10496A0074011200398E518F528552629000C7E04D
:10497A00A851B8000DD395524008E552900044F072
:10498A0080099000C7E014900044F0E56C60067559
:10499A0052007551009000BEE0B4030890003DE05B
:1049AA00655D6002800BA21FB34004D2218002B26F
:1049BA0021E55D640B6005E55DB41D099000B0E07A
:1049CA00600312202B900042E0655D60079000436F
:1049DA00E0B55D03756E00A213B35006A212B3B31D
:1049EA004003024A9490007CE0B401739000FEE018
:1049FA00B40214120C5590006FE075F0BEA4FFAE1D
:104A0A00F08E5B8F5C8056E56675F00A84FF7E0047
:104A1A0090057612621AE0F55A755900AE59AF5AE6
:104A2A009000A1E01261F374648E048F05FF126195
:104A3A00E38C5B8D5CE55C90000EF0AE59AF5A904A
:104A4A00007AE01261F374648E048F05FF1261E349
:104A5A0074BE8C068D071261F38E5B8F5C80179093
:104A6A00007AE075F0BEA4FFAEF08E5B8F5C90001A
:104A7A00A1E090000EF0E560C394CC500690007A55
:104A8A00E070028003123CC7D213E56CB40106E55C
:104A9A005D640B60028009756F019000467401F035
:104AAA00E56C70799000C3E0600D90006EE0A8514B
:104ABA00B800069552400280389000C3E0B402174D
:104ACA0090003BE0655D600790003CE0B55D0375D2
:104ADA006F03756B00800CC200756B00900015E4C3
:104AEA00F0A3F090006EE060067409900045F08033
:104AFA002C90003BE0655D600790003CE0B55D03EB
:104B0A00756F0190003BE0B55D069000467401F0B8
:104B1A0090003CE0B55D067402900046F0A210B326
:104B2A00920EA210B330B601B35003024D08756D50
:104B3A00019000A3E0B43D1975E700A210B3400844
:104B4A00E5B54404F5B58006E5B554FBF5B575E75A
:104B5A0010E5B54401F5B5741C900066F0A21092F8
:104B6A000EE55DD3944A4014D212E55DD3946D40AC
:104B7A000B7404900045F0D222755D469000CBE09C
:104B8A00B40107E569C3941440028009123BF37427
:104B9A0013900045F0A229300301B3501D75E700B8
:104BAA00A229B34008E5B54408F5B58006E5B55431
:104BBA00F7F5B575E710A2299203A22A300401B3CA
:104BCA00501D75E700A22AB34008E5B54402F5B5C1
:104BDA008006E5B554FDF5B575E710A22A9204A240
:104BEA002B300501B3500FA22BB34004D2A0800290
:104BFA00C2A0A22B9205A22C300601B3500FA22C00
:104C0A00B34004D2978002C297A22C9206A22D30FA
:104C1A000701B3500FA22DB34004D2A28002C2A250
:104C2A00A22D9207A22E300801B3500FA22EB34034
:104C3A0004D2A18002C2A1A22E9208A22F30090199
:104C4A00B3501D75E700A22FB34008E5B54440F5FF
:104C5A00B58006E5B554BFF5B575E710A22F9209E0
:104C6A00A230300A01B3501D75E700A230B34008E4
:104C7A00E5B54480F5B58006E5B5547FF5B575E729
:104C8A0010A230920AA231300B01B3500FA231B3F5
:104C9A004004D2878002C287A231920BA232300C22
:104CAA0001B3500FA232B34004D2908002C290A244
:104CBA0032920CE569C394415009740E900045F094
:104CCA00123BF390004DE0FE900049E004C39E4081
:104CDA0009900049E0D39406400974FB900045F01E
:104CEA00123BF3900052E06015900052E0FE9000F3
:104CFA004CE06E600974FE900045F0123BF3A2226C
:104D0A00B34004C296C2959000FBE0600CAE51AF6E
:104D1A00527414BE00059F40028048900083E090C0
:104D2A005A6FF8282873803BA2B4B35005A224B363
:104D3A0040028005123D1FD2248028A2A3B3500549
:104D4A00A225B340028005123D1FD2258015A2A4D8
:104D5A00B35005A223B340028005123D1FD223801F
:034D6A00028000C4
:105A6F00024D30024D32024D45024D58024D6B0230
:025A7F004D6D6B
:104D6D00A215B3B3500890003DE0655D6003024E9F
:104D7D004CA201B35006A200B3B34003024E4890BB
:104D8D0000BEE0B403028003024E1DA20DB34067C6
:104D9D00A221B3402D12363AE55CF5FBE55BF5FC3F
:104DAD00D293A202B34002D2879000DCE0B402108D
:104DBD00123667E55CF5FBE55BF5FC75A700D28760
:104DCD00803312363AE55CF5EBE55BF5ECD291A25A
:104DDD0002B34006E5B54410F5B59000DCE0B40231
:104DED0014123667E55CF5EBE55BF5EC75A700E5B0
:104DFD00B54410F5B5801712363AE55CF5FBE55B69
:104E0D00F5FCE55CF5EBE55BF5ECD293D291802BEF
:104E1D0012363AE55CF5FBE55BF5FCD293A202B3E5
:104E2D004002D2879000DCE0B40210123667E55CD8
:104E3D00F5FBE55BF5FC75A700D287C215D216A26E
:104E4D0016B3B3500890003EE0655D6003024F2B32
:104E5D00A201B35006A200B3B34003024F27900046
:104E6D00BEE0B403028003024EFCA20DB34067A264
:104E7D0021B3402D12363AE55CF5E9E55BF5EAD252
:104E8D0094A202B34002D2909000DCE0B402101262
:104E9D003667E55CF5E9E55BF5EA75A700D290802C
:104EAD003312363AE55CF5EDE55BF5EED292A202F2
:104EBD00B34006E5B54420F5B59000DCE0B402142E
:104ECD00123667E55CF5EDE55BF5EE75A700E5B52A
:104EDD004420F5B5801712363AE55CF5E9E55BF54A
:104EED00EAE55CF5EDE55BF5EED294D292802B12FE
:104EFD00363AE55CF5E9E55BF5EAD294A202B340FA
:104F0D0002D2909000DCE0B40210123667E55CF539
:104F1D00E9E55BF5EA75A700D290D215C216E56FEB
:0E4F2D00905A81F82828730253A29000E3E006
:065A8100024F34024F3712
:104F3B00905AB4F8282873121B078012121B078093
:0E4F4B000D121B918008121C3D8003121C3DAC
:0F5AB400024F42024F47024F4C024F51024F56D2
:104F5900756F020253A2121D69121E80A237B34057
:104F6900229000A5E0F56B900076E0256BFE90009D
:104F790044E075F01E84FC7F00EE2CF5347410902B
:104F89000045F09007AEE0FEA3E0FF740A1261F35A
:104F990090000AE0FCA3E0FD74098F02FF1261E3AF
:104FA9008D078C038E048A058B061260E19007B287
:104FB900EEF0A3EFF09000CCE0B401087478BE00E5
:104FC900059F4002800D74789007B2F8E4F0E8A3D9
:104FD900F0801B9007B2E0FEA3E0FF74F0BE00036F
:104FE9009F500B74F09007B2F8E4F0E8A3F0E534B1
:104FF90070037534019007B2E0FEA3E0FFE5342F9A
:10500900FF50010E9007B2EEF0A3EFF0756F039019
:035019000046E06E
:035A8700024F5F6C
:10501C00905AC3F82828738010A2384003756F0A81
:09502C008007A2384003756F0BE8
:095AC30002502302502502502E6E
:105035000253A29006BDE060031221149000FCE02B
:10504500B401149000FDE0A851B800049552500732
:10505500E55EC3955F400280030250E29000B1E037
:10506500D39402403F900085E02403A851B8000482
:1050750095525009900087E0D3956050028008D280
:10508500017408900045F0900085E0A851B800052E
:10509500D39552500B900087E02403C395605002CE
:1050A500C2018039900085E02403A851B800049519
:1050B500525007E55EC3955F40028008D20174082F
:1050C500900045F0900085E0A851B80005D39552B1
:1050D5005009E55F240FC3955E5002C2019000CBD5
:1050E500E07007E569C3941440028002D201A20171
:1050F5004005756F04800A756F10900015E4F0A3E4
:10510500F0A20DB34029E56675F00A84FF7E009094
:10511500057612621AE0C394695005122060800F6B
:105125009007B0E0F8A3E09007AEC8F0A3C8F0027E
:0651350053A29000B1E05E
:065A8A0002503802513702
:10513B00905ACCF8282873120D3F8012120D3F8025
:0E514B000D120EED8008120F9F8003120F9FB1
:0F5ACC0002514202514702514C025151025156B0
:105159009006C1E060031221F0756F050253A21297
:1051690010AB756F069006C5E060031222E0900649
:10517900C9E060031223BC0253A290000EE060064E
:10518900A20DB3B34002801D90000EE02529FFAEA9
:105199002850010E8E288F29E55DD3941250069070
:1051A900000EE014F01212F1756F079006CDE06061
:1051B900031224989006D1E060031225740253A2C9
:1051C9009000FEE0B40203120CCD12154E756F0863
:1051D9009006D5E060031226509006D9E0600312CC
:1051E900272C0253A212190AA215B35005A216B30D
:1051F90040028004D215D216756F109006DDE0606A
:10520900031228089006E1E060031228E40253A281
:105219000253A2900035E0C394465008C2967446E2
:10522900900035F090003FE0B4011DE534240AF503
:10523900349007B2E0FEA3E0FF740A2FFF50010E7D
:105249009007B2EEF0A3EFF090003FE0B4021DE545
:10525900342414F5349007B2E0FEA3E0FF74142F50
:10526900FF50010E9007B2EEF0A3EFF085345A75A6
:10527900590090003BE0F5721236B2E55C900035BA
:10528900F0900004E559F0A3E55AF0E57290003674
:10529900F0C2189007B2E0F559A3E0F55A90003B27
:1052A900E0F5721236B2E55C900033F0900000E54B
:1052B90059F0A3E55AF0E572900034F0C217E56C95
:1052C900B40105756F0B8003756F030253A290003B
:1052D90039E0C3944650139000CCE0B40104C2965F
:1052E9008002C2957446900039F0900040E0B40104
:1052F9001DE534240AF5349007B2E0FEA3E0FF74FB
:105309000A2FFF50010E9007B2EEF0A3EFF09000C4
:1053190040E0B4021DE5342414F5349007B2E0FEF0
:10532900A3E0FF74142FFF50010E9007B2EEF0A313
:10533900EFF085345A75590090003CE0F572123649
:10534900B2E55C900039F0900006E559F0A3E55A02
:10535900F0E57290003AF0C21A9007B2E0F559A34D
:10536900E0F55A90003CE0F5721236B2E55C900027
:1053790037F0900002E559F0A3E55AF0E572900084
:1053890038F0C219E56CB40103756C00756F0380C0
:09539900088006800480028000F7
:105A90000251680251830251C90251EE02521902A9
:105AA000521C0252D702539A02539C02539E025335
:045AB000A00253A25B
:1053A200900033E0B55D028003025444A2174072BC
:1053B200900000E0FEA3E0FFEF4E6021AE55AF5635
:1053C200900000E0FCA3E0FD120003740A8E048F3B
:1053D20005FF1261E3900000ECF0A3EDF0900034C1
:1053E200E0601A900000E0FEA3E0FFAC55AD56EF7E
:1053F2002DFDEE3CFC900000ECF0A3EDF0900034AB
:10540200E0D39401401A900000E0FEA3E0FFAC5507
:10541200AD56EF2DFDEE3CFC900000ECF0A3EDF05C
:10542200D217AE53AF54900000E0FCA3E0FDEFC3EF
:105432009DEE9C400D123D6CD296C21774C890002E
:1054420033F0A217B3B35007900033E0B55D02808A
:105452000D123D6CD29674C8900033F0C2179000C2
:1054620035E0B55D0280030254FFA218407290003D
:1054720004E0FEA3E0FFEF4E6021AE55AF56900070
:1054820004E0FCA3E0FD120003740A8E048F05FF02
:105492001261E3900004ECF0A3EDF0900036E060BE
:1054A2001A900004E0FEA3E0FFAC55AD56EF2DFDCF
:1054B200EE3CFC900004ECF0A3EDF0900036E0D35B
:1054C2009401401A900004E0FEA3E0FFAC55AD56F3
:1054D200EF2DFDEE3CFC900004ECF0A3EDF0D218B1
:1054E200AE53AF54900004E0FCA3E0FDEFC39DEE89
:1054F2009C400AC2967446900035F0C218A218B3B6
:10550200B35007900035E0B55D02800AC29674463A
:10551200900035F0C218900037E0B55D02800302BA
:1055220055C5A2194072900002E0FEA3E0FFEF4EC3
:105532006021AE55AF56900002E0FCA3E0FD1200E0
:1055420003740A8E048F05FF1261E3900002ECF0EF
:10555200A3EDF0900038E0601A900002E0FEA3E0B4
:10556200FFAC55AD56EF2DFDEE3CFC900002ECF089
:10557200A3EDF0900038E0D39401401A900002E0CD
:10558200FEA3E0FFAC55AD56EF2DFDEE3CFC9000C6
:1055920002ECF0A3EDF0D219AE53AF54900002E04A
:1055A200FCA3E0FDEFC39DEE9C4018123D6C900001
:1055B200CCE0B40104D2968002D295C21974C8908C
:1055C2000037F0A219B3B35007900037E0B55D027F
:1055D2008018123D6C9000CCE0B40104D296800297
:1055E200D29574C8900037F0C219900039E0B55DC9
:1055F200028003025696A21A4072900006E0FEA3B1
:10560200E0FFEF4E6021AE55AF56900006E0FCA3DE
:10561200E0FD120003740A8E048F05FF1261E3900D
:105622000006ECF0A3EDF090003AE0601A9000065C
:10563200E0FEA3E0FFAC55AD56EF2DFDEE3CFC9035
:105642000006ECF0A3EDF090003AE0D39401401A8A
:10565200900006E0FEA3E0FFAC55AD56EF2DFDEE47
:105662003CFC900006ECF0A3EDF0D21AAE53AF541E
:10567200900006E0FCA3E0FDEFC39DEE9C40159078
:1056820000CCE0B40104C2968002C2957446900038
:1056920039F0C21AA21AB3B35007900039E0B55DCF
:1056A2000280159000CCE0B40104C2968002C2953B
:1056B2007446900039F0C21A9000CEE0B402028023
:1056C200030257D6900068E0D39565506490006855
:1056D200E0F4042565FE9000D1E08E00F5F0E88448
:1056E200FF7E008F72EFC39410500CEF8572F0A40E
:1056F200FDACF08D7280037572FF900068E0D39567
:1057020072400B900068E0C39572F570800375706B
:10571200009000ECE0D3957040069000ECE0F5704C
:105722009000EDE0C3957050069000EDE0F57080BA
:1057320071900068E0C39565FE9000D1E08E00F59F
:10574200F0E884FF7E008F72EFC39410500CEF8557
:1057520072F0A4FDACF08D7280037572FF85725AEF
:10576200755900900068E0255AFFAE5950010E8E1F
:10577200598F5A74FFBE0009D39F4005855A708025
:10578200037570FF9000ECE0D3957040069000EC3A
:10579200E0F5709000EDE0C3957050069000EDE0EA
:1057A200F570A20DB3B3500D900069E0FE9000D9E0
:1057B200E0D39E5002800A7407900045F0C29780A1
:1057C2001375A710E5CDC395704004C2978002D22D
:1057D2009775A700E56EC39409500AA2EDB3400580
:1057E200C2ED122C7AAE53AF547498C39F743A9E92
:1057F200400C900067E0C3945A4003025A48A21238
:10580200B34009123BF37406900045F0A21DB34069
:1058120008E5B54404F5B58006E5B554FBF5B5A237
:1058220014B3500EE560D394334007E560C394CCC3
:105832004002802FE5B54401F5B5741C900066F076
:1058420090007AE075F0BEA4FFAEF08E5B8F5C74C0
:1058520002BE000AD39F4006755C02755B00123CD3
:10586200C7D214900067E0D394014007E560C39467
:105872001A40028002C2149006BDE0600312211495
:10588200A229300301B35017A229B34008E5B54459
:1058920008F5B58006E5B554F7F5B5A2299203904F
:1058A20006C1E060031221F0A22A300401B35017AE
:1058B200A22AB34008E5B54402F5B58006E5B55421
:1058C200FDF5B5A22A92049006C5E060031222E01B
:1058D200A22B300501B3500FA22BB34004D2A080FB
:1058E20002C2A0A22B92059006C9E060031223BC5B
:1058F200A22C300601B3500FA22CB34004D29780E1
:1059020002C297A22C92069006CDE0600312249860
:10591200A22D300701B3500FA22DB34004D2A280B2
:1059220002C2A2A22D92079006D1E0600312257452
:10593200A22E300801B3500FA22EB34004D2A18090
:1059420002C2A1A22E92089006D5E0600312265050
:10595200A22F300901B35017A22FB34008E5B54476
:1059620040F5B58006E5B554BFF5B5A22F92099072
:1059720006D9E0600312272CA230300A01B3501777
:10598200A230B34008E5B54480F5B58006E5B554CC
:105992007FF5B5A230920A9006DDE0600312280876
:1059A200A231300B01B3500FA231B34004D2878031
:1059B20002C287A231920B9006E1E060031228E452
:1059C200A232300C01B3500FA232B34004D2908005
:1059D20002C290A232920C900067E0C3945A501017
:1059E200E56EB40909900067E004F0756E00803B33
:1059F200E56EB40903756E00755400755300758D1C
:105A020000758B00756300900066E0C3942A50080D
:105A1200900066E004F08006742A900066F0900020
:105A220066E0B42A06E5B554FEF5B5900067E0D30A
:105A320094014007E569C3944140028009740E90C5
:095A42000045F0123BF30244D7C9
:105ADB000000010001400160018001A001C001E054
:105AEB0002000300039603B603D603F4040005007B
:105AFB000512052405360548055A056C057E0590EB
:105B0B0005A805C005DE0600061406280646066E27
:105B1B0006AE00FF013F015F017F019F01BF01DF67
:105B2B0001FF02FF039503B503D503F303FF04FF46
:105B3B0005110523053505470559056B057D058FB2
:105B4B0005A705BF05DD05F1061306270645066DFE
:105B5B0006AD06ED0FAA0FA50F9F0F9A0F940F8D91
:105B6B000F870F800F780F710F680F600F570F4E55
:105B7B000F450F3B0F300F250F1A0F0E0F020EF5AF
:105B8B000EE80EDB0ECC0EBE0EAE0E9F0E8E0E7DF5
:105B9B000E6C0E5A0E470E340E200E0C0DF70DE246
:105BAB000DCB0DB50D9D0D850D6D0D540D3A0D20C5
:105BBB000D050CE90CCE0CB10C940C760C580C3A70
:105BCB000C1B0BFB0BDB0BBB0B9A0B790B570B3526
:105BDB000B130AF10ACE0AAB0A870A640A400A1CA5
:105BEB0009F809D409B0098C09670943091F08FB97
:105BFB0008D608B2088E086A0846082307FF07DC98
:105C0B0007B9079607730751072F070D06EC06CA4E
:105C1B0006AA068906690649062A060A05EC05CD79
:105C2B0005B0059205750558053C0520050504EAE8
:105C3B0004CF04B5049C0482046904510439042282
:105C4B00040B03F403DE03C803B2039D038903753E
:105C5B000361034D033B03280316030402F202E125
:105C6B0002D102C002B002A002910282027302654D
:105C7B0002570249023C022F02220216020901FDC1
:105C8B0001F201E601DB01D001C601BB01B101A7A5
:105C9B00019D0194018B0182017901700168016002
:105CAB00015801500148014101390132012B0125F5
:105CBB00011E01180111010B010500FF00FA0FA6CF
:105CCB000FA00F990F920F8B0F840F7C0F740F6B1C
:105CDB000F620F580F4E0F430F380F2C0F1F0F1261
:105CEB000F050EF70EE80ED80EC80EB70EA50E93C5
:105CFB000E800E6C0E580E420E2C0E150DFD0DE483
:105D0B000DCB0DB10D950D790D5D0D3F0D200D01D9
:105D1B000CE10CC00C9E0C7C0C590C350C100BEAD6
:105D2B000BC40B9E0B760B4F0B260AFD0AD40AAA4B
:105D3B000A800A550A2A09FF09D409A8097C0950C7
:105D4B00092508F908CD08A10875084A081E07F3AC
:105D5B0007C8079D07730749072006F706CE06A657
:105D6B00067E06570630060A05E405BF059B057738
:105D7B0005540532051004EF04CE04AE048F0471F4
:105D8B0004530435041903FD03E203C703AD039465
:105D9B00037B0363034B0334031E030802F302DE8E
:105DAB0002CA02B602A30291027F026D025C024C90
:105DBB00023C022C021D020E020001F201E401D78B
:105DCB0001CA01BE01B101A6019A018F0185017AB9
:105DDB0001700166015D0153014A01410139013135
:105DEB000129012101190112010B010400FD00F72A
:105DFB0000F000EA00E400DE00D900D300CE00C9B9
:105E0B0000C400BF00BA00B500B100AD00A800A4EB
:105E1B0000A0009C009900950091008E008A0087DD
:085E2B0000840081007E007B71
:10009E007547009007BAE4F0A3F075310075300093
:1000AE00754D00754E00C234D23574FE9007C4F8FB
:1000BE00E4F0E8A3F074FE9007C6F8E4F0E8A3F0CD
:1000CE00745A9007C8F0745A9007C9F0D236C228F5
:1000DE00C238C23322750B00750A00AE0AAF0BACE4
:1000EE0008AD09EDC39FEC9E401674FF1261D375E7
:1000FE00CF01780B740126F6500418E436F650DB67
:10010E0022900041E0B4AA1C900776E0B43C159012
:10011E0007B6E0FEA3E0FFEF4E6009741EBE0004BA
:10012E00D39F500302023D755C00755B0075F809A4
:10013E009007B6E0FEA3E0FF74076F4E6006740EE4
:10014E006F4E7006743A900776F09007B6E0FEA3F5
:10015E00E0FF7408BE001ED39F401A7E017F0890F8
:10016E0007B6E0FCA3E0FD1DBDFF011C1200038ECF
:10017E00598F5A801F9007B6E0FEA3E0FF74081255
:10018E0062378F048E057E017F08CDCCCD12000321
:10019E008E598F5AAE5BAF5C740CD39F74019E5018
:1001AE0003020238A2F9B3407EE55C455B7003752D
:1001BE00A382AE5BAF5C74016F4E700375A300AE8D
:1001CE005BAF5C74026F4E700D9007B7E075F00276
:1001DE00A4FDACF08DA3AE5BAF5C74036F4E7003E9
:1001EE0075A300AE5BAF5C7403BE00039F5013ACEF
:1001FE0059AD5AED2FFFEC3EFE90007212621AE0DE
:10020E00F5A3AE5BAF5CEFB40B09EEB4010574144D
:10021E001261D3AE5BAF5CEFB40B07EEB4010375A6
:10022E00F80D785B1262470201A2900041E4F022C1
:10023E00755C00755B0075F8099007B6E0FEA3E0EB
:10024E00FF7408BE001ED39F401A7E017F089007E0
:10025E00B6E0FCA3E0FD1DBDFF011C1200038E598C
:10026E008F5A801F9007B6E0FEA3E0FF740812625B
:10027E00378F048E057E017F08CDCCCD1200038E04
:10028E00598F5AAE5BAF5C7411D39F74019E5003AD
:10029E0002036EA2F9B3500302036BE55C455B707B
:1002AE000375A3D2AE5BAF5C74016F4E700375A382
:1002BE0000AE5BAF5C74026F4E700D9007B7E075C9
:1002CE00F002A4FDACF08DA3AE5BAF5C74036F4E79
:1002DE00700375A300AE5BAF5C74046F4E70037554
:1002EE00A300AE5BAF5C74056F4E700375A300AEDA
:1002FE005BAF5C74066F4E700375A300AE5BAF5CB4
:10030E0074076F4E700375A300AE5BAF5C74086F1D
:10031E004E700375A300AE5BAF5C7408BE00039F06
:10032E005016AC59AD5AED2FFFEC3EFE90006D12FB
:10033E00621AE5A3F075A300AE5BAF5CEFB41009D3
:10034E00EEB4010574141261D3AE5BAF5CEFB41062
:10035E0007EEB4010375F80D785B12624702029145
:10036E0022755C00755B0075F809AE5BAF5C7417A7
:10037E00BE0004D39F5003020447A2F9B3500302F8
:10038E000444E55C455B700375A3D2AE5BAF5C7451
:10039E00016F4E700375A300AE5BAF5C74026F4EBF
:1003AE00700D9007B7E075F002A4FDACF08DA3AE12
:1003BE005BAF5C74036F4E700375A300AE5BAF5CF6
:1003CE0074046F4E700375A300AE5BAF5C74056F63
:1003DE004E700375A300AE5BAF5C74066F4E700378
:1003EE0075A300AE5BAF5C74076F4E700375A30010
:1003FE00AE5BAF5C74086F4E700375A300AE5BAF5F
:10040E005C7408BE00039F500C90004F12621AE5F8
:10041E00A3F075A300AE5BAF5C74166F4E700574DF
:10042E00141261D3AE5BAF5C74166F4E700375F829
:10043E000D785B12624702037822900041E0B4AB64
:10044E000280030204E2755C00755B0075F809AE6C
:10045E005BAF5C7412BE007CD39F4078A2F9B340B0
:10046E0070E55C455B700375A382AE5BAF5C740197
:10047E006F4E700375A300AE5BAF5C74026F4E706F
:10048E000D9007B7E075F002A4FDACF08DA3AE5B46
:10049E00AF5C74036F4E700375A300AE5BAF5C74FC
:1004AE0003BE00039F500990005412621AE0F5A398
:1004BE00AE5BAF5C74116F4E700574141261D3AEE7
:1004CE005BAF5C74116F4E700375F80D785B126242
:1004DE004702045D229007C1E4F074649007B6F8F9
:1004EE00E4F0E8A3F012036F74C89007B6F8E4F0D6
:1004FE00E8A3F090005BE0B4371A900058E090004B
:10050E004FF0900059E0900050F090005AE09000AB
:10051E0051F080469007C17401F074659007B6F8EB
:10052E00E4F0E8A3F012036F74C89007B6F8E4F095
:10053E00E8A3F090005BE0B4371A900058E090000A
:10054E004FF0900059E0900050F090005AE090006B
:10055E0051F0800674029007C1F09007C2E4F07467
:10056E00669007B6F8E4F0E8A3F012036F74C89033
:10057E0007B6F8E4F0E8A3F090005AE0B437129012
:10058E000058E0900049F0900059E0900052F08041
:10059E00769007C27401F074679007B6F8E4F0E83D
:1005AE00A3F012036F74C89007B6F8E4F0E8A3F056
:1005BE0090005AE0B43712900058E0900049F09045
:1005CE000059E0900052F0803E74029007C2F07421
:1005DE00689007B6F8E4F0E8A3F012036F74C890C1
:1005EE0007B6F8E4F0E8A3F090005AE0B4371290A2
:1005FE000058E0900049F0900059E0900052F080D1
:10060E000674039007C2F022E54E64046006E59975
:10061E0064FF6002802AA2344004D2348020E54E6A
:10062E00600874E6254E900045F0754E00E54D606D
:10063E000874F0254D900045F0754D00C2348002CF
:10064E00C234E54E9033F8F8282873754E00E599BC
:10065E00B4FF03754D01E599B4FE03754D02E5999E
:10066E00B4FD03754D03E599B4FC03754D04E5998E
:10067E00B4FA03754D05E599B4FB06754E01123BB0
:10068E00F3E599B4F906754E04123BF3E599D3944C
:10069E00E54007E599C394F04002801685994F75A1
:1006AE004E027E017F00E54FC394E61261F38E3257
:1006BE008F339007BAE4F0A3F0E599D394C44007C2
:1006CE00E599C394E64002802885994F754E0374D0
:1006DE00E5C3954FF533753200AE32AF33905ADB2A
:1006EE001261C2E493F87401939007BAC8F0A3C8DC
:1006FE00F0D299020AB3900058E070429007BAE027
:10070E00FEA3E0FF74FFBE00039F5009EFC39446A3
:10071E00EE940640119007BAE0FEA3E0FFEFD394EB
:10072E006DEE940640139007BAE0FEA3E0FF900032
:10073E007612621AE599F0800385997380119007FD
:10074E00BAE0FEA3E0FF90007612621AE599F090EF
:10075E0007BA1262019007BAE0FEA3E0FFEFB40100
:10076E0006EEB40702800302089B900776E0B43CC5
:10077E00028003020885C29C900058E0900114F09C
:10078E00900059E0900083F090005AE09000A3F0A2
:10079E0090005BE09000CCF090005CE0900078F070
:1007AE0090005DE09000BEF090005EE09000DCF006
:1007BE0090005FE09000B0F0900060E09000CEF00E
:1007CE00900061E09000FEF012374990006AE090D0
:1007DE0000E5F090006BE090009CF090006CE090D3
:1007EE00009DF074639007B6F8E4F0E8A3F074ABE4
:1007FE00900041F0120448900041E4F075096475D0
:10080E0008001200E3A21C4038757201E572D39401
:10081E0007502CE5729007B6F8E4F0E8A3F074AA3E
:10082E00900041F012010FE572C39407500975094B
:10083E00647508001200E37872740126F650CD80BC
:10084E0036757208E572D3940E502CE5729007B689
:10085E00F8E4F0E8A3F074AA900041F012010FE55D
:10086E0072C3940E50097509647508001200E3787E
:10087E0072740126F650CD74C89007B6F8E4F0E80D
:10088E00A3F0D29C754E00754D007599FB020AB30C
:10089E009007BAE0FEA3E0FFEF4E70068599317522
:1008AE0030009007BAE0FEA3E0FF74016F4E701B9C
:1008BE00AC30AD31AA32AB33ED2BFBEC3AFA8A06F3
:1008CE008B0790007612621AE599F09007BA1262C1
:1008DE00019007BAE0FEA3E0FF74026F4E7021ACE8
:1008EE0030AD3174566D4C7006E54F64E660028093
:1008FE0003123BF3123749854F99754E00754D0023
:10090E00020AB39007BAE0FEA3E0FF9000761262EF
:10091E001AE599F09007BA1262019007BAE0FEA3A9
:10092E00E0FFAC32AD338F028E038C068D07905BE9
:10093E001D1261C2E493F9740193FEEAD39EEB9902
:10094E004009854F99754E00754D00020AB3900708
:10095E00BAE0FEA3E0FF90007612621AE599F090DD
:10096E0007BA1262019007BAE0FEA3E0FFEFB400EF
:10097E0006EEB401028003020AB3900051E075F056
:10098E0002A4FDACF08D72ED900076126225EDFAA8
:10099E00E0FBEA900079126225EBFAE0FBEA2BFA13
:1009AE00900051E0B502028003020AA50DED900001
:1009BE0076126225E572FDE0FAED90007A1262255C
:1009CE00EAFDE0FAEDC39AFD900051E0B505028014
:1009DE0003020AA5E572900078126225E572FDE029
:1009EE00FAED90007B126225EAFDE0FAED2AFD9009
:1009FE000051E0B505028003020AA5E57290007C65
:100A0E00126225FDE0FAED900051E0F4042A900008
:100A1E0058F0E57290007D126225FDE0FAED90002F
:100A2E0051E0F4042A900059F0E57290007E1262B3
:100A3E0025FDE0FAED900051E0F4042A90005AF002
:100A4E00E57290007F126225FDE0FAED900051E014
:100A5E00F4042A9007B6F8E4F0E8A3F074AB900023
:100A6E0041F01204487509647508001200E39007FE
:100A7E00B61262011204487509647508001200E38B
:100A8E009007B61262011204487599F975096475DA
:100A9E0008001200E380FE7599FF75096475080061
:050AAE001200E380FED0
:0F33F80002065902070402089E02091102095C2D
:100AB30022E54D903407F8282873020B989007BA63
:100AC300E0FEA3E0FF90004712621AE0F599900759
:100AD300BA1262019007BAE0FEA3E0FF74116F4EF1
:100AE3007003754D00020B98856D99020B98900762
:100AF300BAE0FEA3E0FF90007612621AE0F599EFE8
:100B0300B40107EEB40703754D009007BA126201F2
:070B1300020B989007BBE004
:0F340700020ABD020AC0020AEB020AF1020B160A
:100B1A009035BAF82828738552998067855E99803E
:100B2A0062856099805D856499805885669980534D
:100B3A00856799804E85689980498569998044902E
:100B4A000016E0F599803CA235B340077599FAC2C0
:100B5A00358017A226B3400575990F800B90004582
:100B6A00E0F599900045E4F0C2268017856A9980DD
:100B7A0012856599800D856B9980087599FC8003AB
:030B8A00754D00A6
:1035BA00020B21020B26020B2B020B30020B3502E7
:1035CA000B3A020B3F020B44020B49020B51020B4E
:0D35DA0076020B7B020B80020B85020B8A30
:0B0B8D009007BA12620180031235E7E6
:03341600020B9511
:100B980022E537255AFFAE5950010E9000761262B1
:100BA8001AE0F538E537255AFFAE5950010E0FBF48
:100BB80000010E90007612621AE0F539853F3BE598
:100BC80038B539058538378041E539D39538401D22
:100BD800E539C39538853AF0A4FFAEF0E53B8E04BD
:100BE8008F05FF1261E3ED2538F537801DE538C321
:100BF8009539853AF0A4FFAEF0E53B8E048F05FFEA
:100C08001261E3EDF4042538F53722E539D3953838
:100C1800401DE539C39538853AF0A4FFAEF0E53BB1
:100C28008E048F05FF1261E3ED2538F537801DE549
:100C380038C39539853AF0A4FFAEF0E53B8E048FB2
:100C480005FF1261E3EDF4042538F5372290007CA6
:100C5800E0B40170E56675F00A84FF7E008F37E521
:100C68006675F00A84ADF07C008D3A753F0A7559B7
:100C780005755A24E537C394115005120B9980065F
:100C88009005ABE0F537E53790006FF0E56675F055
:100C98000A84FF7E008F37E56675F00A84ADF07C24
:100CA800008D3A753F0A755905755A5AE537C39448
:100CB800115005120B9980069005E1E0F537E537EC
:100CC80090000EF02290007CE0B4016AE56675F0B1
:100CD8000A84FF7E008F37E56675F00A84ADF07CE4
:100CE800008D3A753F0A755905755A36E537C3942C
:100CF800115005120B9980069005BDE0F537853730
:100D08004BE56675F00A84FF7E008F37E56675F05F
:100D18000A84ADF07C008D3A753F0A755905755AFD
:100D280048E537C394115005120B9980069005CFFA
:100D3800E0F53785374C22E55E75F00484FF7E00C8
:100D48008F37E55E75F00484ADF07C008D3A753F11
:100D580004755901755A00E537C3943F5005120BC5
:100D68009980069001B5E0F53785372975280090F8
:100D78000044E075F020A4FFAEF09000C7E08E04B8
:100D88008F05FF1261E38D379000AFE0D3955E5079
:100D980003020E459000D3E0D3955E4010ED90011C
:100DA800B6126225E0F52B752A00020E4290009ECD
:100DB800E0D3955E4043E5379001B6126225E0F531
:100DC80038E5379001D6126225E0F5399000D3E076
:100DD800F404255EF53A90009EE0FE9000D3E0F41E
:100DE800042EF53BE538B539058538378003120CF4
:100DF8001385372B752A008041E5379001D612629A
:100E080025E0F538E5379001F6126225E0F53990CE
:100E1800009EE0F404255EF53A9000AFE0FE9000F5
:100E28009EE0F4042EF53BE538B539058538378062
:100E380003120C1385372B752A00020EEC9000D68E
:100E4800E0D3955E5011E537900236126225E0F541
:100E58002B752A00020EEC90009FE0D3955E50435C
:100E6800E537900216126225E0F538E5379002362C
:100E7800126225E0F53990009FE0F404255EF53A0A
:100E88009000D6E0FE90009FE0F4042EF53BE53894
:100E9800B539058538378003120C1385372B752A29
:100EA800008041E5379001F6126225E0F538E53714
:100EB800900216126225E0F5399000AFE0F404259F
:100EC8005EF53A90009FE0FE9000AFE0F4042EF546
:100ED8003BE538B539058538378003120C1385375B
:100EE8002B752A00229000E7E0F53C753F117559F3
:100EF80002755A00AE51AF52E53C75F00FA4FDAC37
:100F0800F0EDD39FEC9E4021E53C8E048F05FF1247
:100F180061E3ED75F010A4FFAEF0E55E75F01184A5
:100F2800FD7C00ED2FF53D800EE55E75F01184FF28
:100F38007E00EF24F0F53D853D37E55E75F01184C0
:100F4800AFF07E008F3A120B9985373EAE51AF5203
:100F58009000E7E075F00FA4FDACF0EDD39FEC9E98
:100F68004028755902755A10853D37120B99853EF0
:100F780038853739AE51AF52E53C8E048F05FF12E4
:100F8800620E8D3A853C3B120C1385372975280073
:100F9800752B64752A00229000E7E0F53C753F1137
:100FA800755902755A00AE51AF52E53C75F00FA461
:100FB800FDACF0EDD39FEC9E4021E53C8E048F05FF
:100FC800FF1261E3ED75F010A4FFAEF0E56075F077
:100FD8001184FD7C00ED2FF53D800EE56075F01164
:100FE80084FF7E00EF24F0F53D853D37E56075F020
:100FF8001184AFF07E008F3A120B9985373EAE51BF
:10100800AF529000E7E075F00FA4FDACF0EDD39F70
:10101800EC9E4028755902755A10853D37120B9978
:10102800853E38853739AE51AF52E53C8E048F0581
:10103800FF12620E8D3A853C3B120C1385372975D9
:1010480028009000B1E0B40453E55E75F00484FF15
:101058007E008F37E55E75F00484ADF07C008D3A34
:10106800753F04755901755A00E537C3943F50051B
:10107800120B9980069001B5E0F537AE28AF29E547
:10108800371261F374648E048F05FF1261E3AE2892
:10109800AF29EF2DFDEE3CFC8C288D29752B64754E
:1010A8002A002290007CE0B40146E56675F00A84C7
:1010B800FF7E008F37E56675F00A84ADF07C008D01
:1010C8003A753F0A755905755A00E537C3941150AA
:1010D80005120B998006900587E0F537AE2AAF2BED
:1010E800E5372FFF50010E74641262378E2A8F2B5A
:1010F80090007DE0B40146E56775F00A84FF7E0044
:101108008F37E56775F00A84ADF07C008D3A753F3E
:101118000A755905755A6CE537C394115005120BB9
:101128009980069005F3E0F537AE2AAF2BE5372F07
:10113800FF50010E74641262378E2A8F2B90008C38
:10114800E0B40249E569C3944175F00584FF7E0067
:101158008F37E56975F00584ADF07C008D3A753FF1
:1011680005755906755A00E537C394135005120BD7
:10117800998006900689E0F537AE2AAF2BE5372F20
:10118800FF50010E74641262378E2A8F2B9000CEA6
:10119800E0B40202800302124AE55E75F01584FF8E
:1011A8007E008F37E55E75F01584ADF07C008D3AD2
:1011B800753F15755903755AF4E537C3940B5005F7
:1011C800120B998006900475E0F537E53775F0FF46
:1011D800A4FFAEF09000CFE08E048F05FF1261E30C
:1011E800ED900068F0E56575F078A4FFAEF074FF47
:1011F8008E048F05FF1261E38C598D5A74028C0698
:101208008D071200398F37AC59AD5A7404FF12623A
:101218000E8D3A753F04755906755A28E537C394FB
:101228001D5005120B9980069006BBE0F537AE2AD3
:10123800AF2BE5372FFF50010E74641262378E2AE8
:101248008F2B90007BE0B4025DE56075F064A4FF2D
:10125800AEF074081200398E5B8F5C74058E048FB3
:1012680005FF1261E38D37AE5BAF5C74058E048FAA
:1012780005FF12620E8D3A753F05755905755ADEE0
:10128800E537C394135005120B998006900667E062
:10129800F537AE2AAF2BE5372FFF50010E746412D5
:1012A80062378E2A8F2B9000BDE0703C900044E09E
:1012B80075F00584FF7E008F37900044E075F005D7
:1012C80084ADF07C008D3A753F05755905755AC097
:1012D800E537C3941D5005120B998006900653E01C
:1012E800F537E537900070F022900084E0B40117DC
:1012F8009007BDE0252BFFAE2A50010E9000D8E0E4
:101308001262378E2A8F2B9000FCE0B401149000F3
:10131800FDE0A851B8000495525007E55EC3955FFB
:10132800400280129000A6E0252BFFAE2A50010E45
:101338008E2A8F2B802F900084E0B40316A228B346
:10134800B350109007C0E0C39405A851B8000695A3
:1013580052400280109000A6E0252BFFAE2A5001D3
:101368000E8E2A8F2B90007EE0B4020280030215B5
:101378004D900081E0602FE566D3944640289000A8
:101388000FE0FEA3E0FF9000BCE075F003A4FDAC05
:10139800F0EFD39DEE9C400E9000E0E0A851B8001D
:1013A80005D39552500302154D9000C9E0855EF0B3
:1013B800A4FFAEF074051261F374071200398E5958
:1013C8008F5A900088E0A851B800049552501290A6
:1013D8000089E075F002A4FDACF0EFC39DEE9C40DF
:1013E8000302154DE55E75F00B84FF7E009006063E
:1013F80012621AFEE0FFEE900080E0FEEF8E008899
:10140800F0A4FFAEF074648E048F05FF1261E38CC4
:10141800598D5A900044E075F018A4FFAEF0900082
:10142800C7E08E048F05FF1261E38C068D079006D6
:101438001E12621AAE59AF5AE01261F374648E0438
:101448008F05FF1261E38C598D5AE564A859B800DD
:1014580077D3955A4072E564C3955AFFE49559FECF
:101468008E598F5A7428BE00039F500C755A2875E0
:101478005900740D900045F0AE59AF5A900081E0C4
:101488001261F374288E048F05FF1261E38C598D65
:101498005AAE28AF29740A8E048F05FF1261E38DB6
:1014A800068C07AC59AD5ACFCECF120003740A8E02
:1014B800048F05FF1261E38C598D5AAE28AF2912AB
:1014C800623F8E288F29807DE564A859B80004956D
:1014D8005A5072AE59AF5AE5641262378E598F5A14
:1014E8007428BE00039F500C755A28755900740D56
:1014F800900045F0AE59AF5A900081E01261F37444
:10150800288E048F05FF1261E38C598D5AAE28AFDF
:1015180029740A8E048F05FF1261E38D068C07ACCF
:1015280059AD5ACFCECF120003740A8E048F05FF2F
:101538001261E38C598D5AAE28AF29EF2DFDEE3C90
:10154800FC8C288D29229000DCE0B4026AE55E75E7
:10155800F00884FF7E008F37E55E75F00884ADF0F3
:101568007C008D3A753F08755901755AE0E537C317
:10157800943F5005120B998006900275E0F5378567
:10158800372D752C00AE2CAF2DAC2AAD2B120003D5
:1015980074648E048F05FF1261E38C2C8D2D9000EE
:1015A80079E08C068D071261F374648E048F05FF51
:1015B8001261E38C2C8D2DAE28AF29AC2AAD2B12ED
:1015C800000374648E048F05FF1261E38C288D2953
:1015D800900079E08C068D071261F374648E048F95
:1015E80005FF1261E38C288D29A20D401DAE51AF75
:1015F800527405BE00039F5002D20DE560D394CC0F
:101608004008D2017411900045F09000DBE0B4026C
:10161800089000DDE0640160028035AE28AF29E55E
:101628006A1261F374E78E048F05FF1261E38C2858
:101638008D299000DCE0B40217AE2CAF2DE56A12BC
:1016480061F374E78E048F05FF1261E38C2C8D2DF6
:1016580090009BE05402601B900092E0A851B800F3
:1016680012D39552400DA20DB3B35007E560C39451
:101678009A40028028AE35AF36900090E075F002AF
:10168800A4FDACF0EF2DFDEE3CFC74022DFD5001E5
:101698000CE560BC0007D39D4003754301856036A7
:1016A800753500E54370030217919000EEE0C3958D
:1016B8004350030217839000FEE0C394025076E57E
:1016C8006675F00A84FF7E0090057612621AE0F5CE
:1016D8005A755900AE59AF5A900091E01261F374EF
:1016E800648E048F05FF1261E38C5B8D5C9000EEC5
:1016F800E004C395438C068D071261F39000EEE079
:101708008E048F05FF1261E38C5B8D5CAE28AF29D8
:10171800EF2DFDEE3CFC8C288D299000DCE0B40216
:1017280012AE2CAF2DAA5BAB5CEF2BFBEE3AFA8A1C
:101738002C8B2D80469000EEE004C39543854BF03A
:10174800A4FFAEF09000EEE08E048F05FF1261E377
:101758008C5B8D5CAE28AF29EF2DFDEE3CFC8C2810
:101768008D299000DCE0B40212AE2CAF2DAA5BAB41
:101778005CEF2BFBEE3AFA8A2C8B2D05439000EE9A
:10178800E0C39543500375430090009BE05401600B
:101798001B90008FE0A851B80012D39552400DA2BB
:1017A8000DB3B35007E55EC394CC4002802590008A
:1017B8008DE075F003A4FFAEF0E5402FFF50010E59
:1017C80074032FFF50010EE55EBE0007D39F400350
:1017D800754401855E40E54470030218C49000EF2B
:1017E800E0C3954450030218B69000FEE0C394028B
:1017F8005076E56675F00A84FF7E009005761262E1
:101808001AE0F55A755900AE59AF5A90008EE01299
:1018180061F374648E048F05FF1261E38C5B8D5C49
:101828009000EFE004C395448C068D071261F39095
:1018380000EFE08E048F05FF1261E38C5B8D5CAED8
:1018480028AF29EF2DFDEE3CFC8C288D299000DC7B
:10185800E0B40212AE2CAF2DAA5BAB5CEF2BFBEE13
:101868003AFA8A2C8B2D80469000EFE004C3954409
:10187800854CF0A4FFAEF09000EFE08E048F05FFDA
:101888001261E38C5B8D5CAE28AF29EF2DFDEE3C39
:10189800FC8C288D299000DCE0B40212AE2CAF2D10
:1018A800AA5BAB5CEF2BFBEE3AFA8A2C8B2D054436
:1018B8009000EFE0C3954450037544009000F1E0B8
:1018C8002529FFAE2850010E8E288F299000A0E010
:1018D800A828B80004952950099000A0E0F52975BA
:1018E80028009000DCE0B4020D9000A0E0A82CB81D
:1018F8000006952D400280099000A0E0F52D752C7A
:1019080000229000DCE0B401028003021A15A20D47
:10191800B35003021A139000A7E0B40168AE28AFD1
:1019280029AC51AD52120003743C8E048F05FF128E
:1019380061E39000B7E0BC00109D400D9000B9E055
:10194800A828B8000495295002D202AE28AF29ACC5
:1019580051AD52120003743C8E048F05FF1261E3EF
:101968009000B7E0C3940ABC0015D39D40119000C5
:10197800B9E0C39405A828B80005D395295002807A
:1019880002C2028068AE28AF29AC51AD52120003E2
:1019980074788E048F05FF1261E39000B7E0BC00F5
:1019A800109D400D9000B9E0A828B8000495295072
:1019B80004D2028038AE28AF29AC51AD52120003D0
:1019C80074788E048F05FF1261E39000B7E0C3942A
:1019D8000ABC0015D39D40119000B9E0C39405A836
:1019E80028B80005D3952950028002C202A202B38A
:1019F8004019AE28AF299000B8E01261F374648EE4
:101A0800048F05FF1261E38C288D298002C202A28F
:101A180000B34006A201B3B35009900015E4F0A347
:101A2800F08024AE28AF297400D39F74019E400C27
:101A3800900015E528F0A3E529F0800B74FF9000CD
:101A480015F8E4F0E8A3F09000BEE0D39402400C4F
:101A58009000A9E07006A20DB3B34002801AAE2828
:101A6800AF2974021261F38E288F29AE2CAF2D7422
:101A7800021261F38E2C8F2D9000A7E0B4011AAEEC
:101A880028AF2974021261F38E288F29AE2CAF2D4E
:101A980074021261F38E2C8F2DAE28AF29745E125A
:101AA80061F3740A8E048F05FF1261E38C288D2977
:101AB8009000DCE0B40217AE2CAF2D745E1261F317
:101AC800740A8E048F05FF1261E38C2C8D2DAE28CD
:101AD800AF297402BE000AD39F40067529027528F3
:101AE80000AE2CAF2D7402BE000AD39F4006752DA0
:101AF80002752C00900013E528F0A3E529F0229048
:101B08000044E0900376126225E0F5417542649046
:101B18000044E0FE9000B2E0D39E4037E55E75F0E9
:101B28000884FF7E008F37E55E75F00884ADF07C91
:101B3800008D3A753F08755903755A96E537C39471
:101B48001F5005120B99800690042BE0F537853756
:101B5800428035E55E75F00884FF7E008F37E55ECC
:101B680075F00884ADF07C008D3A753F087559030F
:101B7800755AB6E537C3941F5005120B9980069025
:101B8800044BE0F537853742229000E8E0F53C75D4
:101B98003F11755904755A00AE51AF52E53C75F0C6
:101BA8000FA4FDACF0EDD39FEC9E4021E53C8E04E4
:101BB8008F05FF1261E3ED75F010A4FFAEF0E55E4E
:101BC80075F01184FD7C00ED2FF53D800EE55E7506
:101BD800F01184FF7E00EF24F0F53D853D37E55E8A
:101BE80075F01184AFF07E008F3A120B9985373E5D
:101BF800AE51AF529000E8E075F00FA4FDACF0EDE7
:101C0800D39FEC9E4028755904755A10853D3712AC
:101C18000B99853E38853739AE51AF52E53C8E0475
:101C28008F05FF12620E8D3A853C3B120C138537E7
:101C380041754264229000E8E0F53C753F11755902
:101C480004755A00AE51AF52E53C75F00FA4FDACD7
:101C5800F0EDD39FEC9E4021E53C8E048F05FF12EA
:101C680061E3ED75F010A4FFAEF0E56075F0118446
:101C7800FD7C00ED2FF53D800EE56075F01184FFC9
:101C88007E00EF24F0F53D853D37E56075F0118461
:101C9800AFF07E008F3A120B9985373EAE51AF52A6
:101CA8009000E8E075F00FA4FDACF0EDD39FEC9E3A
:101CB8004028755904755A10853D37120B99853E91
:101CC80038853739AE51AF52E53C8E048F05FF1287
:101CD800620E8D3A853C3B120C1385374175426480
:101CE8009000E3E0B40479900044E0FE9000B2E094
:101CF800D39E4037E55E75F00884FF7E008F37E598
:101D08005E75F00884ADF07C008D3A753F08755912
:101D180003755A96E537C3941F5005120B99800630
:101D280090042BE0F5378537428035E55E75F0087D
:101D380084FF7E008F37E55E75F00884ADF07C0087
:101D48008D3A753F08755903755AB6E537C3941F20
:101D58005005120B99800690044BE0F53785374201
:101D68002290007CE0B4013BE56675F00A84FF7EB2
:101D7800008F37E56675F00A84ADF07C008D3A7502
:101D88003F0A755905755A12E537C3941150051263
:101D98000B998006900599E0F537E5422537C394FD
:101DA80064F54290007DE0B4013BE56775F00A8474
:101DB800FF7E008F37E56775F00A84ADF07C008DF3
:101DC8003A753F0A755905755A7EE537C39411501F
:101DD80005120B998006900605E0F537E542253790
:101DE800C39464F542E5412542F534900084E0B49B
:101DF80002109007BCE02534FE9000D8E0F4042ED1
:101E0800F5349000DBE0D394014040E56AC394E7E1
:101E1800501D74E7C3956AFE9007BEE08E00F5F08A
:101E2800E884FF7E008F37E5342537F534801CE5DC
:101E38006AC394E7FE9007BEE08E00F5F0E884FFE1
:101E48007E008F37E534C39537F534A20D4006E59B
:101E5800412464F534E534D394644009E534C394EB
:101E680064F53480037534009000B4E0C3953450B1
:101E7800069000B4E0F53422D20090006EE0A8513C
:101E8800B800049552504190006EE0A851B8000483
:101E98009552500375340F90006EE004A851B800B5
:101EA800049552500375340A90006EE02402A8513C
:101EB800B8000495525005753405C20090006EE0D4
:101EC80060067409900045F0C2387E017F009000DA
:101ED800BAE01261F39000C9E08E048F05FF126129
:101EE800E3E55EBC0017D39D40139000C3E0B40245
:101EF80004D2388002C200740A900045F09000BBFA
:101F0800E0C3956650159000CDE0A851B80004953F
:101F1800525002C200740B900045F0E566C3946409
:101F2800501D900113E0600D900113E0A851B80016
:101F380006955240028008C200740B900045F0A23A
:101F48000040037534059000FCE0B401149000FDD6
:101F5800E0A851B8000495525007E55EC3955F406C
:101F68000280089000A5E0F534803A900084E0B43F
:101F78000306A228B3B34002802B9007C0E0C394A5
:101F880005A851B800049552500C9000A5E0F5340E
:101F9800740C900045F09007C0E0A851B800049573
:101FA800525002C20085346B900076E02534FE90D2
:101FB8000044E075F01E84FC7F00EE2CF53422907E
:101FC8000044E075F00584FF7E008F37900044E000
:101FD80075F00584ADF07C008D3A753F05755903A1
:101FE800755AD69000C7E01475F00584FF7E00E5A9
:101FF80037BE00039F5005120B99800BE5379004FC
:102008004C126225E0F537E5379007BFF09007BF1F
:10201800E0FE9000B6E0C39E50089000B6E090073E
:10202800BFF022E56675F00A84FF7E0090057612FF
:10203800621AE0F546E546D394644010E546C39439
:102048006475F00F84FF7E008F468003754600900C
:102058000099E02546F546229007B0E0FEA3E0FF90
:102068007404120039E55E1261F3740F8E048F0553
:10207800FF1261E39007AEECF0A3EDF090008CE066
:10208800B40262E569C3944175F00584FF7E008F50
:1020980037E56975F00584ADF07C008D3A753F052C
:1020A800755906755A14E537C394175005120B99DC
:1020B800800690069DE0F5379007AEE0FEA3E0FFAE
:1020C800740A8E048F05FF1261E3E5378C068D07CD
:1020D8001261F3740A8E048F05FF1261E39007AE54
:1020E800ECF0A3EDF09007AEE0FEA3E0FF9007B49C
:1020F800E0FCA3E0FDEDD39FEC9E400F9007B4E019
:10210800F8A3E09007AEC8F0A3C8F0229006BDE09F
:10211800903419F8282873804C85527280479000B3
:10212800C9E0855EF0A4FFAEF074081200398F7222
:102138008033856072802E856672802985677280FB
:1021480024856872801F856972801A856A72801575
:102158008565728010856472800B856B728006902D
:052168000016E0F57215
:1034190002211F02212102212602213A02213F0213
:10342900214402214902214E02215302215802213D
:073439005D02216202216720
:10216D009006BEE0FE9006BFE0D39E404B9006BDAC
:10217D00E0B404189006BFE0C395725002D22990C6
:10218D0006BEE0D395724002C229802A9006BEE0B9
:10219D00C3957250099006BFE0D39572500280022C
:1021AD00D2299006BEE0D3957250099006BFE0C3C8
:1021BD0095725002C229802A9006BEE0D3957240D6
:1021CD00099006BFE0C3957240028002C2299006B5
:1021DD00BEE0C3957240099006BFE0D395724002F0
:1021ED00D229229006C1E0903440F8282873804C03
:1021FD0085527280479000C9E0855EF0A4FFAEF075
:10220D0074081200398F728033856072802E856656
:10221D007280298567728024856872801F85697236
:10222D00801A856A7280158565728010856472804A
:0C223D000B856B728006900016E0F572B5
:103440000221FB0221FD02220202221602221B029D
:10345000222002222502222A02222F0222340222C4
:073460003902223E02224363
:102249009006C2E0FE9006C3E0D39E405F9006C1AF
:10225900E0B404189006C3E0C395725002D22A90E4
:1022690006C2E0D395724002C22A803E9006C2E0BF
:10227900C3957250099006C3E0D39572500280024B
:10228900D22A9006C2E0D3957250099006C3E0C3E2
:1022990095725002C22A9006C1E0B401099000D596
:1022A900E0D3956050028002C22A802A9006C2E0DB
:1022B900D3957240099006C3E0C39572400280022B
:1022C900C22A9006C2E0C3957240099006C3E0D3C2
:1022D90095724002D22A229006C5E0903467F82808
:1022E9002873804C85527280479000C9E0855EF062
:1022F900A4FFAEF074081200398F728033856072C2
:10230900802E85667280298567728024856872802F
:102319001F856972801A856A7280158565728010B9
:10232900856472800B856B728006900016E0F572E9
:103467000222EB0222ED0222F202230602230B02C2
:10347700231002231502231A02231F0223240223E7
:073487002902232E0223336A
:102339009006C6E0FE9006C7E0D39E404B9006C5C6
:10234900E0B404189006C7E0C395725002D22B90EE
:1023590006C6E0D395724002C22B802A9006C6E0D9
:10236900C3957250099006C7E0D395725002800256
:10237900D22B9006C6E0D3957250099006C7E0C3E8
:1023890095725002C22B802A9006C6E0D3957240FE
:10239900099006C7E0C3957240028002C22B9006DD
:1023A900C6E0C3957240099006C7E0D39572400212
:1023B900D22B229006C9E090348EF8282873804CDD
:1023C90085527280479000C9E0855EF0A4FFAEF0A7
:1023D90074081200398F728033856072802E856689
:1023E9007280298567728024856872801F85697269
:1023F900801A856A7280158565728010856472807D
:0C2409000B856B728006900016E0F572E7
:10348E000223C70223C90223CE0223E20223E7024C
:10349E0023EC0223F10223F60223FB022400022472
:0734AE000502240A02240FAD
:102415009006CAE0FE9006CBE0D39E404B9006C9DD
:10242500E0B404189006CBE0C395725002D22C900C
:1024350006CAE0D395724002C22C802A9006CAE0F3
:10244500C3957250099006CBE0D395725002800275
:10245500D22C9006CAE0D3957250099006CBE0C302
:1024650095725002C22C802A9006CAE0D39572401C
:10247500099006CBE0C3957240028002C22C9006FB
:10248500CAE0C3957240099006CBE0D3957240022D
:10249500D22C229006CDE09034B5F8282873804CD4
:1024A50085527280479000C9E0855EF0A4FFAEF0CA
:1024B50074081200398F728033856072802E8566AC
:1024C5007280298567728024856872801F8569728C
:1024D500801A856A728015856572801085647280A0
:0C24E5000B856B728006900016E0F5720B
:1034B5000224A30224A50224AA0224BE0224C302D4
:1034C50024C80224CD0224D20224D70224DC0224FB
:0734D500E10224E60224EBF2
:1024F1009006CEE0FE9006CFE0D39E404B9006CDF5
:10250100E0B404189006CFE0C395725002D22D902A
:1025110006CEE0D395724002C22D802A9006CEE00D
:10252100C3957250099006CFE0D395725002800294
:10253100D22D9006CEE0D3957250099006CFE0C31C
:1025410095725002C22D802A9006CEE0D39572403A
:10255100099006CFE0C3957240028002C22D900619
:10256100CEE0C3957240099006CFE0D39572400248
:10257100D22D229006D1E09034DCF8282873804CCB
:1025810085527280479000C9E0855EF0A4FFAEF0ED
:1025910074081200398F728033856072802E8566CF
:1025A1007280298567728024856872801F856972AF
:1025B100801A856A728015856572801085647280C3
:0C25C1000B856B728006900016E0F5722E
:1034DC0002257F02258102258602259A02259F025C
:1034EC0025A40225A90225AE0225B30225B8022582
:0734FC00BD0225C20225C735
:1025CD009006D2E0FE9006D3E0D39E404B9006D10C
:1025DD00E0B404189006D3E0C395725002D22E9049
:1025ED0006D2E0D395724002C22E802A9006D2E028
:1025FD00C3957250099006D3E0D3957250028002B4
:10260D00D22E9006D2E0D3957250099006D3E0C336
:10261D0095725002C22E802A9006D2E0D395724058
:10262D00099006D3E0C3957240028002C22E900637
:10263D00D2E0C3957240099006D3E0D39572400263
:10264D00D22E229006D5E0903503F8282873804CC1
:10265D0085527280479000C9E0855EF0A4FFAEF010
:10266D0074081200398F728033856072802E8566F2
:10267D007280298567728024856872801F856972D2
:10268D00801A856A728015856572801085647280E6
:0C269D000B856B728006900016E0F57251
:1035030002265B02265D02266202267602267B02E3
:10351300268002268502268A02268F022694022608
:073523009902269E0226A377
:1026A9009006D6E0FE9006D7E0D39E404B9006D523
:1026B900E0B404189006D7E0C395725002D22F9067
:1026C90006D6E0D395724002C22F802A9006D6E042
:1026D900C3957250099006D7E0D3957250028002D3
:1026E900D22F9006D6E0D3957250099006D7E0C351
:1026F90095725002C22F802A9006D6E0D395724077
:10270900099006D7E0C3957240028002C22F900655
:10271900D6E0C3957240099006D7E0D3957240027E
:10272900D22F229006D9E090352AF8282873804CB8
:1027390085527280479000C9E0855EF0A4FFAEF033
:1027490074081200398F728033856072802E856615
:102759007280298567728024856872801F856972F5
:10276900801A856A72801585657280108564728009
:0C2779000B856B728006900016E0F57274
:10352A0002273702273902273E022752022757026B
:10353A00275C02276102276602276B02277002278F
:07354A007502277A02277FBA
:102785009006DAE0FE9006DBE0D39E404B9006D93A
:10279500E0B404189006DBE0C395725002D2309085
:1027A50006DAE0D395724002C230802A9006DAE05C
:1027B500C3957250099006DBE0D3957250028002F2
:1027C500D2309006DAE0D3957250099006DBE0C36B
:1027D50095725002C230802A9006DAE0D395724095
:1027E500099006DBE0C3957240028002C230900674
:1027F500DAE0C3957240099006DBE0D3957240029A
:10280500D230229006DDE0903551F8282873804CAF
:1028150085527280479000C9E0855EF0A4FFAEF056
:1028250074081200398F728033856072802E856638
:102835007280298567728024856872801F85697218
:10284500801A856A7280158565728010856472802C
:0C2855000B856B728006900016E0F57297
:1035510002281302281502281A02282E02283302F3
:10356100283802283D02284202284702284C022816
:073571005102285602285BFD
:102861009006DEE0FE9006DFE0D39E404B9006DD51
:10287100E0B404189006DFE0C395725002D23190A3
:1028810006DEE0D395724002C231802A9006DEE076
:10289100C3957250099006DFE0D395725002800211
:1028A100D2319006DEE0D3957250099006DFE0C385
:1028B10095725002C231802A9006DEE0D3957240B3
:1028C100099006DFE0C3957240028002C231900692
:1028D100DEE0C3957240099006DFE0D395724002B5
:1028E100D231229006E1E0903578F8282873804CA7
:1028F10085527280479000C9E0855EF0A4FFAEF07A
:1029010074081200398F728033856072802E85665B
:102911007280298567728024856872801F8569723B
:10292100801A856A7280158565728010856472804F
:0C2931000B856B728006900016E0F572BA
:103578000228EF0228F10228F602290A02290F027E
:10358800291402291902291E02292302292802299D
:073598002D02293202293740
:10293D009006E2E0FE9006E3E0D39E404B9006E168
:10294D00E0B404189006E3E0C395725002D23290C1
:10295D0006E2E0D395724002C232802A9006E2E090
:10296D00C3957250099006E3E0D395725002800230
:10297D00D2329006E2E0D3957250099006E3E0C39F
:10298D0095725002C232802A9006E2E0D3957240D1
:10299D00099006E3E0C3957240028002C2329006B0
:1029AD00E2E0C3957240099006E3E0D395724002D0
:1029BD00D23222AE2EAF2F74F5D39F74019E4008F4
:1029CD00782E126247022ADA752F01752E00AE514C
:1029DD00AF52E546BE000DD39F40099000ABE0D34A
:1029ED00954740028023754700E546C39552F57221
:1029FD009000AEE0D395454008E5452572F545803C
:102A0D00069000AEE0F54580020547900087E0D3C3
:102A1D009560401CE55EC3955F4015AE51AF52E524
:102A2D0046BE00039F50099000ACE0D3954840028C
:102A3D00806E9007C3E0A851B800049552500375FD
:102A4D004A009007C3E0A851B8000BD39552400639
:102A5D00E5529007C3F0E54A7041E552C39546F53E
:102A6D0072E572D3940540037572059000ADE0C315
:102A7D0095455007E572C3954540028009E545C36C
:102A8D009572F54580069000ADE0F5459000ADE0FE
:102A9D00D3954540069000ADE0F5457548008002A0
:102AAD000548E54A7016900087E0C39560500DE526
:102ABD00462405A851B8000695524002800F90009B
:102ACD009AE0F545754A0174789007C3F022AE2E51
:102ADD00AF2F74E9D39F74039E4008782E1262477E
:102AED00022C79752F01752E00754532A233402ABF
:102AFD0075451990009AE075F002A4FFAEF0E54718
:102B0D00BE0006D39F4002D2330547754A03747841
:102B1D009007C3F0754900022C68AE51AF52E546DF
:102B2D006F4E7003022C68E546BE000DD39F400921
:102B3D009000ABE0D395474002800F754700E54A02
:102B4D00C394035003754519800DE546C39552F5A1
:102B5D0072E5472572F547900087E0D39560400EEA
:102B6D009007C3E0A851B80007D395524002800CDE
:102B7D00054990009AE0B54903754A00E54AB4034A
:102B8D0006A20DB3B34002800A0549E549B43C03E2
:102B9D00754A02E54AB402299007C3E0A851B8006E
:102BAD000ED395524009E5529007C3F07549009038
:102BBD000087E0C39560500975490074789007C38C
:102BCD00F0E54A705A900087E0D39560401CE55EB1
:102BDD00C3955F4015AE51AF52E546BE00039F5001
:102BED00099000ACE0D39548400280087548007507
:102BFD00454B8028E552C39546F572E572D3940591
:102C0D004003757205900087E0D395604008E54854
:102C1D002572F5488006E5482406F548754900E516
:102C2D004A7016900087E0C39560500DE546240567
:102C3D00A851B80006955240028003754A01E54A35
:102C4D00B40118754519054990009AE0B549067506
:102C5D004A0275490074789007C3F0E54575F00A8E
:102C6D00A4FFAEF09007B8EEF0A3EFF022E56E9062
:102C7D00359FF828287390007FE07003022E28906E
:102C8D0000B5E0B401028003022D78900042E0B55A
:102C9D005D028003022D757E017F00E5BE1261F39A
:102CAD00E5BD2FFF50010E8E598F5A74101261F32E
:102CBD0090006DE08E048F05FF1261E39007C4EC68
:102CCD00F0A3EDF0E56A60089000DBE064026002BD
:102CDD0080269000DDE0B4011F9007C4E0FEA3E064
:102CED00FF74E71261F3E56A8E048F05FF1261E34D
:102CFD009007C4ECF0A3EDF090007FE0B4022790B4
:102D0D0007C6E0FEA3E0FF9007C4E0FCA3E0FDEFE3
:102D1D002DFDEE3CFC74018C068D071200399007D9
:102D2D00C4EEF0A3EFF09007C4E0FEA3E0FF900720
:102D3D00C6E0FCA3E0FDEDD39FEC9E4004D23680AF
:102D4D0002B2369007C4E0F8A3E09007C6C8F0A31E
:102D5D00C8F09000B1E064016006A236B3B3400242
:102D6D0080069007C5E0F55E022E26D2367E017FE5
:102D7D0000E5BE1261F3E5BD2FFF50010E8E598F98
:102D8D005A74101261F390006DE08E048F05FF12DE
:102D9D0061E39007C4ECF0A3EDF0E56A60089000E4
:102DAD00DBE06402600280269000DDE0B4011F903C
:102DBD0007C4E0FEA3E0FF74E71261F3E56A8E0439
:102DCD008F05FF1261E39007C4ECF0A3EDF09000C6
:102DDD007FE0B402279007C6E0FEA3E0FF9007C492
:102DED00E0FCA3E0FDEF2DFDEE3CFC74018C068DA7
:102DFD00071200399007C4EEF0A3EFF09007C4E07E
:102E0D00F8A3E09007C6C8F0A3C8F09000B1E06445
:102E1D000160069007C5E0F55E8003755E009000C9
:102E2D007BE07006756E01022C7A75BB180233F3C8
:102E3D0090007BE07003022FC97E017F00E5BE127A
:102E4D0061F3E5BD2FFF50010E8E598F5A9000C1D1
:102E5D00E0B4010F7E0F7FFFAC59AD5A12623F8E69
:102E6D00598F5A9000E6E0B40245AE59AF5A900022
:102E7D001FE0FCA3E0FDEDD39FEC9E400A90001FE8
:102E8D00E559F0A3E55AF0AE59AF5A900021E0FC98
:102E9D00A3E0FDEFD39DEE9C400A900021E559F093
:102EAD00A3E55AF0AE59AF5A74041200398F6090F1
:102EBD0000E6E0704CAE59AF5A90001FE0FCA3E065
:102ECD00FDEFD39DEE9C400912623F8E598F5A80C3
:102EDD0006755A00755900AE59AF5A74101261F348
:102EED0090006AE08E048F05FF1261E38C598D5AB4
:102EFD0074FFBC0009D39D4005855A608003756041
:102F0D00FE9000B1E0B401028003022FC7A20DB301
:102F1D00B3500E900085E0A851B80005D3955250DE
:102F2D0003022FBC900086E075F019A4FFAEF0905F
:102F3D0000C9E08E048F05FF1261E39000C2E085A9
:102F4D0060F0A4FFAEF074648D028C038E048F05C7
:102F5D00FF1261E3EA2DFDEB3CFC8C598D5AE56ABD
:102F6D00600F9000DBE0B402089000DDE0640160CA
:102F7D00028017AE59AF5A74E71261F3E56A8E04F9
:102F8D008F05FF1261E38C598D5AAE59AF5A9007D8
:102F9D00C4E0FCA3E0FDEDD39FEC9E4005855A5E99
:102FAD00800BA236B340069007C5E0F55E800BA2FC
:102FBD0036B340069007C5E0F55E8003756000905E
:102FCD00007EE07006756E02022C7A75BB19023315
:102FDD00F390007EE0700302307EE55DD3955040A6
:102FED000302307C90001DE0FEA3E0FFE564126259
:102FFD003790001DEEF0A3EFF07E017F00E5BE12CD
:10300D0061F3E5BD2FFF50010E8E598F5A9000EBE5
:10301D00E07013740A1261F374518E048F05FF1260
:10302D0061E38D648019AE59AF5A740A1261F38F42
:10303D00048E057E017F95CDCCCD1260E18F64E5C8
:10304D0064D39464400375646490001DE0FEA3E0B6
:10305D00FFE5642FFF50010E90001DEEF0A3EFF081
:10306D00900082E0048E048F05FF1261E38D648071
:10307D00037564329000CEE07006756E03022C7AF3
:10308D0075BB130233F39000CEE0604A7E017F00E2
:10309D00E5BE1261F3E5BD2FFF50010E8E598F5A1B
:1030AD0074041200398F659000D0E08565F0A4FDA1
:1030BD00ACF07464FF1261E38D659000CFE085651F
:1030CD00F0A4FFAEF074FF8E048F05FF1261E3EDE7
:1030DD00900069F0800375650090007CE0700675C6
:1030ED006E04022C7A75BB170233F390007CE0B4AA
:1030FD000102800302318C7E017F00E5BE1261F377
:10310D00E5BD2FFF50010E8E598F5A9007C8E06014
:10311D00199007C8E014905B5F12008CE493FC7467
:10312D000193FDEDC39FEC9E400280069007C8E021
:10313D0014F09007C8E0C394B3501DAE59AF5A9028
:10314D0007C8E004905B5F12008CE493FC7401935C
:10315D00FDEFC39DEE9C400280069007C8E004F091
:10316D009007C8E0FE9000A2E08E0088F0A4FFAEAC
:10317D00F074648E048F05FF1261E38D6680037514
:10318D00660090007DE07006756E05022C7A75BBA9
:10319D00160233F390007DE0B40102800302323554
:1031AD007E017F00E5BE1261F3E5BD2FFF50010EDC
:1031BD008E598F5A9007C9E060199007C9E0149095
:1031CD005CC912008CE493FC740193FDEDC39FEC7C
:1031DD009E400280069007C9E014F09007C9E0C335
:1031ED0094B3501DAE59AF5A9007C9E004905CC915
:1031FD0012008CE493FC740193FDEFC39DEE9C4093
:10320D000280069007C9E004F09007C9E0FE900027
:10321D00A8E08E0088F0A4FFAEF074648E048F05D4
:10322D00FF1261E38D67800375670075BB1F023365
:10323D00F37E017F00E5BE1261F3E5BD2FFF500166
:10324D000E8E598F5A74091261F374E68E048F0530
:10325D00FF1261E38D69900084E07006756E0702C0
:10326D002C7A75BB150233F3900084E070030233A2
:10327D008F7E017F00E5BE1261F3E5BD2FFF50018A
:10328D000E8E598F5A74041200398F68900084E0A5
:10329D00B401159000D8E08568F0A4FFAEF0740776
:1032AD00120039EF9007BDF0900084E0B402159044
:1032BD0000D8E08568F0A4FFAEF07407120039EF76
:1032CD009007BCF0900084E0B40302800302338DBC
:1032DD009000C5E070389000D8E0601CE568C3949C
:1032ED00195002D228E568D394644002C228900098
:1032FD00A4E09007C0F08014E568C394195002D281
:10330D0037E568D394324002C237C22880639000FB
:10331D00A4E070349000D8E08568F0A4FFAEF0749E
:10332D00FF8E048F05FF1261E3ED9007C0F0AE51E3
:10333D00AF52741EBE0006D39F4002D228E560D363
:10334D0094E54002C2288029E568C3940A500DAE69
:10335D0051AF52741EBE0004D39F50028002D2287A
:10336D00E560D394E54002C2289000A4E09007C028
:10337D00F09007C0E0C39405500674059007C0F0A7
:10338D0080037568009000DBE07006756E08022CF6
:10339D007A75BB1480509000DBE060397E017F00B0
:1033AD00E5BE1261F3E5BD2FFF50010E8E598F5A08
:1033BD00EFD39421EE940E4005756AFF8015AE593A
:1033CD00AF5A74101261F374E38E048F05FF12610E
:1033DD00E38D6A8003756A0090007FE0600575BB20
:0633ED001A800375BB18F5
:10359F00022C83022E3D022FDE0230930230F802FE
:0B35AF0031A102323E0232750233A34C
:0533F300056ED2EC2282
:096225002582F582500205832256
:0F008C0025E050020583258250020583F582226C
:1061C200EF2F500205832582F582E5833E2EF5836B
:0161D20022AA
:10623700CFC39FFF50011E22C3EF9DFFEE9CFE229E
:086247000806B6000218062249
:0D620100A3E004F07006120049E004F02252
:0E003900048007C3CE13CECF13CFD5E0F6223E
:1060E100BC000FBE0008ED8FF084FFADF022E4FE8E
:1060F100FF22BE000DEF60FE54F0606F20E7030247
:106101006197EAC0E0EBC0E078017A0075F001EE3A
:1061110020E710EF25E0FFEE33FE0AC5F023C5F0BE
:1061210030E7F0EA5407F9096A7A007B0060010858
:10613100C3EC9E40167004ED9F4010ED9FFDEC9E58
:10614100FCE5F0CA4ACA03F5F08005E5F003F5F075
:10615100C3EE13FEEF13FFD9D77908CACBCAD8D043
:10616100EAFEEBFFD0E0FBD0E0FA22EC8FF084FCFA
:10617100ED54F045F0C48FF084FEEDC454F045F0C9
:10618100C48FF084FDEEC4FE54F02DFFEE540F3C9D
:10619100FEADF07C0022790078008FF0EC7E0820C3
:1061A100E70DC3CD33CD33C933C9C833C8DEF0845D
:1061B10049F9E5F08FF0BE00E6FD7C00E9FFE8FE5D
:0161C10022BB
:0E61F300F88FF0A4FFE5F0CE88F0A42EFE2277
:10000300EF8DF0A4F9A8F0EF8CF0A428F8EE8DF0B2
:06001300A428FEE9FF2213
:1061D300600D782B0261DD007830D8FED5E0F8221F
:1061E300EEC0E07E001260E1EFFDEEFCD0E0FE22A7
:0C620E00EEC0E07E001260E1D0E0FE2255
:03001B0002001EC2
:0300530002005652
:03009B00020071EF
:0300000002622E6B
:09622E0075817475D000023E6711
:0B621A00E5822FF582E5833EF583222C
:0A0049000582D5820215831582227C
:10001E00C0E0C0F0C083C082C0D075D000123DA138
:0B002E00D0D0D082D083D0F0D0E032E0
:10005600C0E0C0F0C083C082C0D075D000123DA4FD
:10006600D0D0D082D083D0F0D0E032C0E0C0F0C093
:1000760083C082C0D075D000123E29D0D0D082D0A5
:0600860083D0F0D0E0324F
:00000001FF
